:03000000021105E5
:03000B000200A54B
:03002B000202AE20
:03005B0002045F3D
:030073000204394B
:1000800002030406080C10182030406080040608A3
:100090000C10182030406080A0C00D0D0403060D28
:1000A0000503030202C2AFC0D0C0E020620C20688A
:1000B00002419D306602415DE47385258AC262E596
:1000C00025F4700221242068022111207210758B02
:1000D00000D0E0D0D0C292C290C291D2AF32C292D0
:1000E000C290C2917406D5E0FDE53C1420E21520D3
:1000F000E10D207D02D293307D02D295020121D202
:1001000094020121207D02D295307D02D29302011A
:1001100021758B00D0E0D0D0C292C290C291D2AFF4
:1001200032758B00D0E0D0D0D2AF32419DE5256052
:100130000A207D02D292307D02D290C291419DE58B
:10014000256002D291207D02C290307D02C2924190
:100150009DE525600A207D02D290307D02D292205A
:100160007D02C292307D02C290419D207D02C295E7
:10017000307D02C293207D02C293307D02C295740D
:1001800006D5E0FDE525600A207D02D292307D0291
:10019000D290C291419D207D02C295307D02C293D2
:1001A000C2947406D5E0FDE525600A207D02D29256
:1001B000307D02D290C291419DC294207D02C295B1
:1001C000307D02C2937406D5E0FDE5256002D29130
:1001D000207D02C290307D02C292419DC294207D5A
:1001E00002C293307D02C2957406D5E0FDE525601C
:1001F00002D291207D02C290307D02C292419D20A8
:100200007D02C293307D02C295C2947406D5E0FD92
:10021000E525600A207D02D290307D02D292207DB9
:1002200002C292307D02C290419D207D02C2933075
:100230007D02C295207D02C295307D02C293740674
:10024000D5E0FDE525600A207D02D290307D02D206
:1002500092207D02C292307D02C290419D30723D5B
:10026000E53C20E21A20E129207D02C295307D0282
:10027000C293207D02C293307D02C29502029D206E
:10028000E1E6207D02C295307D02C293C294020253
:100290009DC294207D02C293307D02C295E525F473
:1002A000F58A758B00D262D0E0D0D0D2AF32C2AF27
:1002B000C2AD53E6EFC0D0C0E0D2D3D2AFC2CEE5DC
:1002C0002960072074461529610C78007900E580C3
:1002D000307E01F430E70278FF53DACF207E03430B
:1002E000DA20307E0343DA10C2D8C271E580307E56
:1002F00001F430E70279FFC3E89970CE30610375ED
:1003000029402074037529408859D270E52A600479
:10031000152A611C20740543DA01C2D820700261DD
:1003200044A859206102C270207402612D882230D5
:10033000690AC3E522955E4003855E227882B60491
:1003400003852224C3E52594404002D26420CF0CCB
:10035000D0E0D0D0C2D343E610D2AD32C2CF7802C3
:10036000E52960053074021529C3E559940140055B
:10037000755C006186755D00756400E55C2401F5BF
:100380005C5003755CFF7982B7020EE547601EC3BF
:10039000E522943240178546227982B7030FE5475C
:1003A000600BC3E52294324004798E8722C3E52393
:1003B000952260084004152361BC0523D8C8056454
:1003C000E56470021564D565647565017805C3E55B
:1003D0006495664058C3E564956750087801756573
:1003E000030203F0C3E56495685005780175650163
:1003F000C3E55F9524401F7982B704028122E54757
:10040000701485245FE56404600385666475650186
:1004100075233C02042DE55F285005755FFF81229E
:10042000F55FE55F047006755DFF7564FFD0E0D091
:10043000D0C2D343E610D2AD32C0D0C0E0C2AF5379
:10044000917F53E67FC260759100C3E49550F594A7
:10045000E49551F595759104D0E0D0D0D2AF32C279
:10046000AF53E6EFC2ADC0D0C0E0C0F0D2D3D2AF40
:0E047000A8FBA9FCC2D830710281C653DACFB6
:10047E00207E0343DA10307E0343DA20D271E5800A
:10048E00307E01F420E702819D88268927C19D5385
:10049E00DACF207E0343DA20307E0343DA10C2D84F
:1004AE00C271307402C1897800E580307E01F4306B
:1004BE00E702C1898859C17053DACF207E0343DA2F
:1004CE0020307E0343DA10C271206102A19653DA06
:1004DE00CF207E0343DA10307E0343DA20C2D8D217
:1004EE007188548955C3E89552F8E99553F9E4FBA0
:1004FE007E027A00C3E8948CE9940050057558008A
:10050E00A186C3E894C8E994005008E4D2E4FB7ACB
:10051E000AA163C3E89468E994015008E4D2E3FBAE
:10052E007A0FA163C3E894D0E994025008E4D2E2B2
:10053E00FB7A1EA163C3E894A0E994055008E4D2A7
:10054E00E1FB7A3CA163C3E89498E994085008E46F
:10055E00D2E0FB7A787E00C3E89556FCE99557FD0C
:10056E0030E708ECF42401FCEDF4FD755800C3EC03
:10057E009AED9E500375580188568957A854A9556F
:10058E00885289537802C170C3E89526F8E99527F9
:10059E00F9307C02C154307B02C154307A02C14D15
:1005AE00207502A1B9E9FDE8FCA1D8E9C313F9E869
:1005BE0013F8307902C14DE9C313F9E813F8307816
:1005CE0002C14DE9C313FDE813FC206126C3EC9470
:1005DE001CED94024002A1EFED7018C3EC94C850CC
:1005EE00120528C3E528940A5002C189755900D214
:1005FE0070C189E528600215287400207F03789663
:10060E00E624FAFEE43400FFC3EC9EFCED9FFD50A1
:10061E000678007900C154C3EC94FFED94004006B7
:10062E0078FF7900C154EC856FF0A4C5F0A2F733C2
:10063E00F87900400302067078FF7900020670E92F
:10064E00C313F9E813F8307C0EE9600278FFC3E8B3
:10065E001338F8E43400F9C3E894FFE9940040023B
:10066E0078FF8859D270206102C189741FF4552F0A
:10067E004BF52FC274E42B7002D27475294030747E
:10068E000375290A306102C19D20740353DAFE7589
:10069E002A20307403752A0AD0F0D0E0D0D0C2D30D
:1006AE00D2AD43E6103279010206D279030206D2A8
:1006BE00790A0206D2791E0206D279640206D2792E
:1006CE00C80206D27817E4D5E0FDD8FAD9F6227A18
:1006DE00147B780206F97A107B8C0206F97A0D7B70
:1006EE00B40206F97A0B7BC80206F9AC2575250112
:1006FE007902B27DE4C294D5E0FDE5256002D29187
:10070E00D5E0FDC291D5E0FDD294D5E0FDE52560A2
:10071E000A207D02D292307D02D290E570D5E0FDA6
:10072E00207D02C292307D02C2907496D5E0FDD932
:10073E00C1EAF8D5E0FDD8FBDBB1C2948C2522C30B
:10074E007C007D0075F00005F0EA33FAEB33FB50C8
:10075E00F6EB13FBEA13FAC3E9FFE8FEE89AF8E9B1
:10076E009BF95004EFF9EEF8B3EC33FCED33FDD505
:10077E00F0DFEDF9ECF822E889F08A20D2D4F8A95E
:10078E00F07B0030F70B7BFFF42401F8E9F4340022
:10079E00F9E88520F0A4ADF0F8E98520F0A4AFF0DB
:1007AE00FEED2EF974003FFA7C04C3EA13FAE91346
:1007BE00F9E813F8DCF48BF030F70AE8F42401F8CA
:1007CE00E9F43400F9E889F0C2D4F8A9F02278826D
:1007DE00B6040302087EC3E5599419401FE52D5453
:1007EE00067019E547703878057994E71460077834
:1007FE000A1460027812C3E53B984020E547600971
:10080E0085615F7564FF756501852224E4F53EF50B
:10081E003FF540F541F542F54702087E75470179EF
:10082E0094E7147013E523F43333F913F8E9540104
:10083E0004F9E854FE020872E714147014E523F468
:10084E00333333F913F8E9540304F9E854FC02087E
:10085E007AE523F433333333F913F8E954070404F8
:0E086E00F9E854F8C39440F8E99400F9883E84
:10087C00893F22E547603BC3E53B13F9E53A13F8A2
:10088C00C3E53E98F8E53F99F9500CC3E89480E92C
:10089C0094FF40160208BAC3E8947FE99400500311
:1008AC000208BA787F79000208BA788079FF884309
:1008BC00894422E5476058E5432540F8E544354135
:1008CC00F9854420E4300701F43542FA30E709C3D6
:1008DC00EA94F040150208FCC3EA940F5003020896
:1008EC00FC78FF79FF7A0F0208FC780079007AF027
:1008FC00C3E524955E5006E52460092115E54420E6
:10090C00E70D2115E54430E706884089418A4222EB
:10091C00E547700302098078A1E6FAC3E54333F892
:10092C00E54433F9120785E930E70BC3E89480E915
:10093C0094FF40132157C3E8947FE994005002219F
:10094C0057787F79002157788079FFE820E715C325
:10095C00E52398F84009C3E89401400302097E7826
:10096C000102097EE8F424012523F8400302097EE4
:10097C0078FF884522E54770030209E378A2E6FA7E
:10098C00A841A942120785E930E70CC3E89401E9B4
:10099C0094FF40160209BAC3E894FFE9940050038F
:1009AC000209BA78FF79000209BA780179FFE920C7
:1009BC00E715C3E54598F84009C3E89401400302E4
:1009CC0009E178000209E1E8F424012545F8400327
:1009DC000209E178FF88242278FFC264E52D5406D1
:1009EC00702FD264C3E53B940A4009C3E5259440BB
:1009FC005002C264E53B601974FF853BF084853777
:100A0C00F0A4F8C5F0600278FFC3E895615002A825
:100A1C00618860227883E6F520120F2175E8901228
:100A2C0006B475E890E5E820ECFBA8BDA9BE120F52
:100A3C00A1756B2C756C00C3740013FD742C13FC26
:100A4C00742C2CFC74003DFDECFAEDFBC3E89AE928
:100A5C009B4014E56B242CF56BE56C3400F56CEACB
:100A6C002CFAEB3DFB80E5AE6BAF6CC3E56C13F978
:100A7C00E56B13F8C3E913F9E813F8E56B28F5698E
:100A8C00E56C39F56A7A03C3E913F9E813F8DAF778
:100A9C00AA201A7009756B00756C00020ABA1AEA62
:100AAC006008EE28FEEF39FFDAF88E6B8F6C22753A
:100ABC00E890227883E6FFE5E820ECF7A8BDA9BE14
:100ACC00056DC3E56D94084052756D00E9FA79A087
:100ADC00E76044EA7007E56E601B020AF5C3E8950F
:100AEC006E6010E56E5006600C14020B010460F988
:100AFC00020B01E56EF56EC3946D401B755EC0C3B1
:100B0C0094044013755E80C39404400B755E40C31F
:100B1C0094044003755E0075BB0622EFC39401601C
:100B2C001BC3E894FFE994035012C3E8956BE99555
:100B3C006C5009E55E600C155E020B4FE55EF460CF
:100B4C0002055EA85EC3E524985002A824C3E8956C
:100B5C005F400AA85FE55FF46003855F5E8825E56A
:100B6C006DB4070375BB1022743279A387F0A4C54A
:100B7C00F0A2F733F8C3E8955E4002A85E8822889D
:100B8C00248825886122753A00753B7F2275C82020
:100B9C00A8CCA9CD75C824AA38AB3988388939C3F3
:100BAC00E89AF8E99BF9AA3AAB3BAC3AAD3B7E0428
:100BBC007F02C3EB940440021E1FC3EB9408400257
:100BCC001E1FC3ED13FDEC13FCDEF7C3EA9CFAEB1E
:100BDC009DFBEF6009C3E913F9E813F8DFF7EA2886
:100BEC00FAEB39FB8A3A8B3B400122753AFF753B95
:100BFC00FF2230600261FE854C50854D51D260431E
:100C0C00E680227892E6FFC3E535948240010FC35B
:100C1C00E53594A040010FC3EF940640027F057E9A
:100C2C00021E3072010EC3E53B940350060E0E30CB
:100C3C0072010EC3E53B940250060E0E3072010E8B
:100C4C00A93BA83A7A04C3E913F9E813F8DAF7C315
:100C5C00E89EF8E99400F94009C3E89402E994008D
:0F0C6C0050047802E4F9E9FBE8FAC3E913FDE864
:100C7B0013FC884C894DC3EF94036037EF20E00DD4
:100C8B00E82CF8E93DF9ECFAEDFB020CABE828F89F
:100C9B00E939F9C3E89402F8E99400F97A02E4FB24
:100CAB00C3EF9403400D8A4E8B4F884889498C4A79
:100CBB008D4B22884E894F8A488B498C4A8D4B220B
:100CCB0030600281CBD26043E680E52D540660276D
:100CDB00A83AA93BE53494085006E820E002A94D58
:100CEB00759100C3E498F594E499F595759104D248
:100CFB006053917F43E68022D265753D00752000DD
:100D0B00020D16D265753D00752040E52D54066029
:100D1B0002C265D2AF206005E53D60012278017A01
:100D2B0002C3E53B940540027802C3E53B940A40BD
:100D3B00027803C3E53B940F40027A0330690478D1
:100D4B001E7A01206007E53D6003D2AF22D2AF00CF
:100D5B0000C2AFC3E53BFB940F40027B0FEB0430AB
:100D6B0073012320620123F93069027982E58BC379
:100D7B009940D0053DEAFBE59BF45440B52004DBDC
:100D8B00F6A1B2206502A116C265759100AE3AAF0D
:100D9B003BC3E49EF594E49FF595759104D26053A3
:100DAB00917F43E680A116306502A116D895D2AF8C
:100DBB002230690B0534206016753400020DDA20E1
:100DCB00600D20650A206B07158115810215C12264
:100DDB00A84EA94F75910053917FC3E498F594E405
:100DEB0099F595759104854850854951D26043E634
:100DFB00802278003064053065027801E53575F0A6
:100E0B0007A4F9E5F028F5F0E9A2F013A2F113A27B
:100E1B00F213F535C394785003753578C3E53595E2
:100E2B00364008D266C292C290C291306002C1367F
:100E3B00854A50854B51D26043E68022C2AFC295A2
:100E4B00C293C29430720B9001FF7406D5E0FD0281
:100E5B000E5D207D02D295307D02D293759F117568
:100E6B003C02020F9CC2AF207D02C290307D02C2B9
:100E7B00923072179001DCC294207D02C293307DB8
:100E8B0002C2957406D5E0FD020E9990013F3062C7
:100E9B0006E5256002D291207D03759F01307D030D
:100EAB00759F21753C03020F9CC2AFC295C293C2C2
:100EBB009430720B9001B97406D5E0FD020ECA2076
:100ECB007D02D293307D02D295207D03759F213018
:100EDB007D03759F01753C04020F9CC2AFC291301C
:100EEB007217900196207D02C295307D02C293C28B
:100EFB00947406D5E0FD020F0790012D30620EE5CC
:100F0B0025600A207D02D292307D02D290759F110E
:100F1B00753C05020F9CC2AFC295C293C29430724E
:100F2B000B90016B7406D5E0FD020F37D294207D38
:100F3B0003759F01307D03759F21753C06020F9C45
:100F4B00C2AF207D02C292307D02C29030721F90E0
:100F5B00022A207D02C295307D02C293207D02C2FF
:100F6B0093307D02C2957406D5E0FD020F7C900193
:100F7B005130620EE525600A207D02D290307D0251
:100F8B00D292207D03759F21307D03759F01753CA7
:100F9B0001C266D2AF2290012BC292C290C291C203
:100FAB0095C293C294C262227880760708760708AE
:100FBB0076010876040876FF0876FF08760908762E
:100FCB0002087601087601788C760108760008769F
:100FDB00B40876FF0876FF0876FF0876030876FFDD
:100FEB000876010876FF0876250876D0087678080B
:100FFB0076C80876040876FF08760108760008762E
:10100B007A08760A087601227887E6FFC272BF0358
:10101B0002D2727888C27DE630E102D27DC27E7840
:10102B0089E630E102D27EC3EF94026008758E012F
:10103B00D273021045758E00C273227880E614902D
:10104B0000809378A1F67881E6149000809378A2C3
:10105B00F6120FA1227886E61490008D9378A3F6F2
:0F106B00120FA122789FE6F8700108C3E89411D4
:10107A0040027811E82828F5662566256628F5676E
:10108A0025662828F56822789CE67536FF75370CA0
:10109A00B402067536A075370AB40306753682752A
:1010AA00370522227896E6FA7897E6FB307F047AAB
:1010BA00007BFFC3EB9AFCC3948250027C82756F5B
:1010CA0000056FEC856FF0A4C3E5F0948040F2222E
:1010DA00D27F11AE1206C37A007B007C101206B9C9
:1010EA00E5592AFA74003BFBDCF37C04C3EB13FBDF
:1010FA00EA13FADCF7FEC27F11AE22E5EF20E6031F
:10110A007520000520903FFFE520146006901DFF22
:10111A001460009304600375EF12C2D353D9BF75EC
:10112A0081C043FF801206B475EF0243B203E5B3F0
:10113A00240420E702F5B3120FA17580FF75A400FD
:10114A0075F19175D47F75900075A53F75F23F755D
:10115A00D50075A60175E241120FB31215FC7898F5
:10116A008670C2AF1206CD1206DD1206C31206E45D
:10117A001206C31206EB1206C312171F1206CD126D
:10118A0006CD1206C8C2AFE4F8F6D8FD78C879C809
:10119A00308707D9FBD8F7021C00120FB31215FCCF
:1011AA00111311461160116F119111AD11AE78989A
:1011BA008670120FA175885075891275C8247591A9
:1011CA000475D84075A82275B80275E690759B809B
:1011DA00759D0075D10E75BC5875BB0675BA11752B
:1011EA00E8801206B4D2AF120A2043DA01C2D8C28A
:1011FA00711206CD753001D2617B037A0CE5587005
:10120A00067A0CDB02218F1206C3207002218FC2DC
:10121A0070E559C3940240E3E52F541F855B5AF5E4
:10122A005BB55AD7DAD7C26153DACF207E0343DAE5
:10123A0020307E0343DA10C2D8C271C27575280005
:10124A001206C8307409C3E528940A4002D27512FE
:10125A0006B978023074027800C3E5599840F0C2A2
:10126A00AF1206DD1206DD1206DDD2AF1206CD750B
:10127A0046001206B9788CE6C39401500302135053
:10128A00E530C394015003021350207435C3E55965
:10129A0094FF5003021350C2AF1206F2D2AF1206E5
:1012AA00C8C3E559940150EFC2AF1206DD1206BE5B
:1012BA001206DDD2AF1206C8C3E55994FF40E9020F
:1012CA0017A47F05D27F11AE1206C8C2AFC27F1122
:1012DA00AEAE59C3E559947FD2AF40741206B4C278
:1012EA00AF1206F2D2AFDFDC11DAC3EE94057897BB
:1012FA00F61206CD12163E1217277F0AD27F11AEBA
:10130A001206C8C2AFC27F11AEAE59C3E559947F67
:10131A00D2AF50E61206B4C2AF1206DD1206BE12F2
:10132A0006DDD2AFDFD611DAEE24057896F612067C
:10133A00CD12163E1217561206C811AEC3E55994BD
:10134A00FF40F40217A4C3E5599546400385594660
:10135A001206C878017988E7B403027805C3E5590B
:10136A00984002417CC2AF1206F21206F21206F24D
:10137A00D2AF1206CD753000E4F531F5320531E50C
:10138A0031F470390532789AE67819146012783295
:10139A0014600D787D14600878FA146003753200C1
:1013AA00C3E53298401715327531B478998670C200
:1013BA00AF1206F2D2AF789886701206C81206BE2D
:1013CA00E5297005307402218F78012074027806AD
:1013DA00C3E5599840A71206C8E5297002218FC2B1
:1013EA00AF120FA1E4F522F523F524F525D2AF7843
:1013FA00858662F53EF53FF540F541F542F56DF516
:10140A0047F52CF52DF535120B92756D0875BB1045
:10141A001206B4120ABBE5E820ECFBA8BDA9BEE996
:10142A007001F8886E120ABF756D0875BB1078874F
:10143A00E6FE760211137887EEF6C2AF755EFF12EA
:10144A000B7485225E85225F852260D2AF752201E8
:10145A00752401752501855D64756501D268D269B7
:0F146A00753400120F21120F4B120B92120B99B7
:10147900120C0F02148A120FA11113756D0075BB9E
:1014890006120D0E120DBC120DDB1207DC120DFD3A
:10149900120E47120B99120BFE120C0F120CCB12E3
:1014A9000D03120DBC120DDB12087F1209E4120D97
:1014B900FD120E70120B99120BFE120C0F120CCBAF
:1014C900120D0E120DBC120DDB1208BF120DFD120A
:1014D9000EB4120B99120BFE120C0F120CCB120D3B
:1014E90003120DBC120DDB12091C120DFD120EE6C2
:1014F900120B99120BFE120C0F120CCB120D0E12BD
:101509000DBC120DDB120981120DFD120F21120BF8
:1015190099120BFE120C0F120CCB120D03120ABBFF
:10152900120DBC120DDB120ABF120DFD120F4B1268
:101539000B99120BFE120C0F120CCB30692F206B7A
:101549002C85615E85615F855D6475650179327A97
:101559000AC3E534994009C269D26A8A3302157609
:10156900C3E5599401400302148A0215C1306A1B6C
:10157900206B18E533147004C26A817FF533C3E523
:10158900599401400302148A0215C1C3E55C940110
:10159900400985615F855D64756501C3E55C94FA01
:1015A9005016307404E529600FC3E53B78F0306BC1
:1015B900027860985002818AC2AF120FA17887E63B
:1015C900FE760211137887EEF6E4F522F523F52469
:1015D900F525F562C268D2AF1206B4120FA13074B4
:1015E90006E5297002218F788DE6C39401400241F6
:1015F900596182901A0D7820121680E520B4A50C45
:10160900A3121680E520B45A0302161E120FB31254
:10161900163E02163D901A0378807B0A121680A3A3
:1016290008DBF9901A0F788C7B15121680A308DB5A
:10163900F9901A2422C2AF1216BF121699901A00F5
:10164900740D121685A37402121685A3741312164B
:1016590085901A0378807B0A121684A308DBF99017
:101669001A0F788C7B15121684A308DBF91216D28F
:101679001216B0901A2422E493F622E6438F0153FE
:101689008FFD75EF0275B7A575B7F1F0538FFE227F
:10169900438F02438F0175EF0275B7A575B7F190B6
:1016A9001A0DF0538FFC22901A0D74A5D185901A4A
:1016B9000E745AD185227A3079D07820901A40D187
:1016C90080E520F709A3DAF7227A3079D0901A4019
:1016D900E7D18509A3DAF922AB71A872BB010279B6
:1016E90080BB02027981BB03027982BB040279942F
:1016F900BB05027983BB06027986BB07027992BBD7
:1017090008027987BB0902799CBB0A027988BB0B5D
:10171900027989E8F7227C051206CDDCFB22C2AFEB
:101729001206DD1206E41206EB1206F21206BE12CA
:1017390006DD1206E41206EB1206F21206BE1206C6
:10174900DD1206E41206EB1206F2D2AF22C2AF1284
:1017590006F21206EB1206E41206DD1206BE1206A6
:10176900F21206EB1206E41206DD1206BE1206F2AA
:101779001206EB1206E41206DDD2AF22AE71AF7289
:10178900C2AF1206DD1206DD1206DD1206BEDEF25A
:101799001206F21206BEDFF8D2AF22F127F11FF1CD
:1017A9001F757101757201757300F1857C05AD595D
:1017B9001206CDC3ED955970F5C3E5599401400A58
:1017C900C3E55994FF40320217E0D1E1D13EF12738
:1017D900C2AF75EF12F11FDCD50573C3E57394032E
:1017E900500280C6F11F0572E5711490009A93F8B2
:1017F90008C3E57298500280AE12171F12171F0511
:1018090071C3E571940C5002809A120FB312163EFF
:08181900C2AF75EF1212171F98
:101A00000D021307070104FFFF09020101A55A0196
:101A100000B4FFFFFF03FF01FF25D078C804FF01DA
:051A200000FF0A01FFB8
:101A40002358503335415357232020202020202075
:101A500023424C48454C4923463333302320202031
:101A60002020202020202020202020202020202076
:101C0000C2AFC2D353D9BF7581C043B20343FF8073
:101C1000752438752503B1BF75EF0275E24043F1B5
:101C20008053A47FD287780379E67C1075220075F3
:101C30002300901DCC7B0675249875250130870202
:101C4000813D208708D8FBD9F9DCF781AD308708C2
:101C5000D8FBD9F9DCF781ADB17FE493A3C39A60D7
:101C6000028126DBDDB171600281267B08E493FAF4
:101C7000A3B152DBF87A30B152752200752300B15E
:101C800071EAFCEBFDC3ED94FE400EB1718A278B27
:101C900028ED30E0048A828B83B1717AC270D8C398
:101CA000ED94FE601050CEBD0022EC600675200061
:101CB0000200008100A827A9280809D804D90281B8
:101CC000C9B175EA89AAF281BB0D8199C3ED94036C
:101CD0005049EDA2E092007AC5C3E5829400E58305
:101CE000941C5093200010438F02438F0175B7A5B9
:101CF00075B7F1F030001FA827A9280809438F0104
:101D0000538FFDD804D902A11689AAE275B7A5752B
:101D1000B7F1F0A3A103538FFC81757AC1BD030C09
:101D2000E493A3FAB136DCF8B12E81758177AA224B
:101D3000AB23B152EBFAEA6222752608C3E52313FE
:101D4000F523E52213F52250066323A0632201D573
:101D500026EAB1BFB1BF75260AEAF4200102D28794
:101D6000300102C287B1BFC3134002C201D526EBC6
:101D700022B175EAFB208702A175308702A17A752E
:101D80002608AE24AF25C3EF13FFEE13FEB1C3B197
:101D9000BFC3EA133087024480FA30E703632201AD
:101DA000C3E52313F523E52213F52250066323A090
:101DB000632201D526D9E52265236523F52222AECB
:101DC00024AF250E0FDEFEDFFCD20122424C486517
:0A1DD0006C6934373132F33006013C
:00000001FF
